******************************************************************************
                  TI ARM Linker PC v20.2.1                     
******************************************************************************
>> Linked Wed Jan  6 14:24:42 2021

OUTPUT FILE NAME:   <enet_tcpecho_server.out>
ENTRY POINT SYMBOL: "_c_int00_noargs"  address: 00006999


MEMORY CONFIGURATION

         name            origin    length      used     unused   attr    fill
----------------------  --------  ---------  --------  --------  ----  --------
  FLASH                 00000000   00100000  00007794  000f886c  R  X
  SRAM                  20000000   00040000  0001db03  000224fd  RW X


SEGMENT ALLOCATION MAP

run origin  load origin   length   init length attrs members
----------  ----------- ---------- ----------- ----- -------
00000000    00000000    00007798   00007798    r-x
  00000000    00000000    00000200   00000200    r-- .intvecs
  00000200    00000200    00007260   00007260    r-x .text
  00007460    00007460    000002dc   000002dc    r-- .const
  00007740    00007740    00000058   00000058    r-- .cinit
20000000    20000000    0001db08   00000000    rw-
  20000000    20000000    00017a93   00000000    rw- .bss
  20017a98    20017a98    00005000   00000000    rw- .stack
  2001ca98    2001ca98    00001070   00000000    rw- .data


SECTION ALLOCATION MAP

 output                                  attributes/
section   page    origin      length       input sections
--------  ----  ----------  ----------   ----------------
.intvecs   0    00000000    00000200     
                  00000000    00000200     startup_ccs.obj (.intvecs)

.text      0    00000200    00007260     
                  00000200    0000079c     lwiplib.obj (.text:tcp_receive)
                  0000099c    000003b4     lwiplib.obj (.text:tcp_process)
                  00000d50    000003a8     lwiplib.obj (.text:tcp_input)
                  000010f8    000002e4     lwiplib.obj (.text:tcp_write)
                  000013dc    000002c8     lwiplib.obj (.text:tcp_slowtmr)
                  000016a4    00000251     ustdlib.obj (.text:uvsnprintf)
                  000018f5    00000001     --HOLE-- [fill = 0]
                  000018f6    00000002     startup_ccs.obj (.text:FaultISR)
                  000018f8    00000228     lwiplib.obj (.text:dhcp_parse_reply)
                  00001b20    0000020c     pinout.obj (.text:PinoutSet)
                  00001d2c    00000200     driverlib.lib : sysctl.obj (.text:SysCtlClockFreqSet)
                  00001f2c    000001ee     uartstdio.obj (.text:UARTvprintf)
                  0000211a    00000002     startup_ccs.obj (.text:IntDefaultHandler)
                  0000211c    000001d8     lwiplib.obj (.text:ip_input)
                  000022f4    000001c0     lwiplib.obj (.text:udp_input)
                  000024b4    00000190     enet_tcpecho_server.obj (.text:main)
                  00002644    0000018c     lwiplib.obj (.text:tcp_output)
                  000027d0    00000184     lwiplib.obj (.text:icmp_input)
                  00002954    0000016c     driverlib.lib : gpio.obj (.text:GPIOPadConfigSet)
                  00002ac0    00000150     lwiplib.obj (.text:etharp_arp_input)
                  00002c10    00000148     lwiplib.obj (.text:tcp_close_shutdown)
                  00002d58    00000140     lwiplib.obj (.text:tivaif_receive)
                  00002e98    0000013c     lwiplib.obj (.text:pbuf_alloc)
                  00002fd4    00000124     lwiplib.obj (.text:dhcp_create_msg)
                  000030f8    0000011c     lwiplib.obj (.text:etharp_output)
                  00003214    00000114     lwiplib.obj (.text:etharp_query)
                  00003328    00000114     lwiplib.obj (.text:tcp_listen_input)
                  0000343c    00000110     enet_tcpecho_server.obj (.text:echo_recv)
                  0000354c    00000100     lwiplib.obj (.text:tivaif_transmit)
                  0000364c    000000f8     lwiplib.obj (.text:mem_malloc)
                  00003744    000000ec     lwiplib.obj (.text:lwIPInit)
                  00003830    000000e8     lwiplib.obj (.text:mem_trim)
                  00003918    000000e0     lwiplib.obj (.text:etharp_find_entry)
                  000039f8    000000dc     lwiplib.obj (.text:etharp_raw)
                  00003ad4    000000d4     lwiplib.obj (.text:autoip_tmr)
                  00003ba8    000000d4     lwiplib.obj (.text:dhcp_select)
                  00003c7c    000000d0     lwiplib.obj (.text:tcp_alloc)
                  00003d4c    000000cc     lwiplib.obj (.text:dhcp_recv)
                  00003e18    000000c8     lwiplib.obj (.text:dhcp_bind)
                  00003ee0    000000c4     lwiplib.obj (.text:InitDMADescriptors)
                  00003fa4    000000c4     lwiplib.obj (.text:dhcp_discover)
                  00004068    000000c4     lwiplib.obj (.text:udp_sendto_if)
                  0000412c    000000c0     lwiplib.obj (.text:tcp_output_segment)
                  000041ec    000000bc     lwiplib.obj (.text:tivaif_hwinit)
                  000042a8    000000b8     lwiplib.obj (.text:tcp_create_segment)
                  00004360    000000b0     lwiplib.obj (.text:lwIPServiceTimers)
                  00004410    000000ac     lwiplib.obj (.text:ethernet_input)
                  000044bc    000000ac     lwiplib.obj (.text:tcp_enqueue_flags)
                  00004568    000000a8     lwiplib.obj (.text:dhcp_release)
                  00004610    000000a8     lwiplib.obj (.text:dhcp_start)
                  000046b8    000000a8     lwiplib.obj (.text:ip_output_if)
                  00004760    0000009c     rtsv7M4_T_le_v4SPD16_eabi.lib : memcpy_t2.asm.obj (.text)
                  000047fc    0000009c     lwiplib.obj (.text:tcp_listen_with_backlog)
                  00004898    00000098     lwiplib.obj (.text:dhcp_reboot)
                  00004930    00000094     enet_tcpecho_server.obj (.text:lwIPHostTimerHandler)
                  000049c4    00000092     lwiplib.obj (.text:pbuf_copy)
                  00004a56    00000002     startup_ccs.obj (.text:NmiSR)
                  00004a58    00000090     lwiplib.obj (.text:tcp_abandon)
                  00004ae8    0000008c     lwiplib.obj (.text:tcp_zero_window_probe)
                  00004b74    00000084     lwiplib.obj (.text:lwIPLinkDetect)
                  00004bf8    00000084     lwiplib.obj (.text:tcp_timewait_input)
                  00004c7c    00000080     lwiplib.obj (.text:dhcp_rebind)
                  00004cfc    00000080     lwiplib.obj (.text:dhcp_renew)
                  00004d7c    00000080     lwiplib.obj (.text:lwIPEthernetIntHandler)
                  00004dfc    00000080     lwiplib.obj (.text:lwIPPrivateInit)
                  00004e7c    00000080     lwiplib.obj (.text:tcp_bind)
                  00004efc    0000007e     lwiplib.obj (.text:autoip_arp_reply)
                  00004f7a    00000002     rtsv7M4_T_le_v4SPD16_eabi.lib : div0.asm.obj (.text)
                  00004f7c    0000007c     lwiplib.obj (.text:dhcp_handle_ack)
                  00004ff8    0000007c     lwiplib.obj (.text:dhcp_timeout)
                  00005074    0000007c     lwiplib.obj (.text:tcp_oos_insert_segment)
                  000050f0    0000007c     lwiplib.obj (.text:tcp_parseopt)
                  0000516c    0000007c     lwiplib.obj (.text:tcp_rst)
                  000051e8    0000007c     lwiplib.obj (.text:tivaif_process_phy_interrupt)
                  00005264    0000007a     rtsv7M4_T_le_v4SPD16_eabi.lib : memset_t2.asm.obj (.text)
                  000052de    00000002     --HOLE-- [fill = 0]
                  000052e0    00000074     lwiplib.obj (.text:etharp_update_arp_entry)
                  00005354    00000074     lwiplib.obj (.text:raw_input)
                  000053c8    00000070     lwiplib.obj (.text:mem_free)
                  00005438    00000070     lwiplib.obj (.text:tcp_fasttmr)
                  000054a8    0000006c     lwiplib.obj (.text:icmp_send_response)
                  00005514    0000006c     lwiplib.obj (.text:memp_init)
                  00005580    00000068     driverlib.lib : interrupt.obj (.text:IntEnable)
                  000055e8    00000068     rtsv7M4_T_le_v4SPD16_eabi.lib : copy_decompress_lzss.c.obj (.text:decompress:lzss:__TI_decompress_lzss)
                  00005650    00000068     lwiplib.obj (.text:dhcp_decline)
                  000056b8    00000068     lwiplib.obj (.text:lwip_standard_chksum)
                  00005720    00000068     lwiplib.obj (.text:netif_set_ipaddr)
                  00005788    00000068     lwiplib.obj (.text:sys_timeout)
                  000057f0    00000068     lwiplib.obj (.text:tcp_output_alloc_header)
                  00005858    00000068     lwiplib.obj (.text:tcp_process_refused_data)
                  000058c0    00000068     lwiplib.obj (.text:udp_bind)
                  00005928    00000066     lwiplib.obj (.text:pbuf_copy_partial)
                  0000598e    00000064     lwiplib.obj (.text:pbuf_header)
                  000059f2    00000002     --HOLE-- [fill = 0]
                  000059f4    00000060     uartstdio.obj (.text:UARTStdioConfig)
                  00005a54    00000060     lwiplib.obj (.text:plug_holes)
                  00005ab4    0000005c     lwiplib.obj (.text:mem_init)
                  00005b10    0000005c     lwiplib.obj (.text:tcp_pcb_remove)
                  00005b6c    0000005a     lwiplib.obj (.text:pbuf_realloc)
                  00005bc6    00000002     --HOLE-- [fill = 0]
                  00005bc8    00000058     driverlib.lib : emac.obj (.text:EMACPHYConfigSet)
                  00005c20    00000058     lwiplib.obj (.text:autoip_create_addr)
                  00005c78    00000058     lwiplib.obj (.text:autoip_start)
                  00005cd0    00000058     lwiplib.obj (.text:memp_malloc)
                  00005d28    00000058     lwiplib.obj (.text:tcp_new_port)
                  00005d80    00000056     lwiplib.obj (.text:tcp_rexmit)
                  00005dd6    00000052     lwiplib.obj (.text:tcp_pbuf_prealloc)
                  00005e28    00000052     lwiplib.obj (.text:tivaif_process_transmit)
                  00005e7a    00000002     --HOLE-- [fill = 0]
                  00005e7c    00000050     driverlib.lib : sysctl.obj (.text:SysCtlPeripheralReset)
                  00005ecc    00000050     uartstdio.obj (.text:UARTwrite)
                  00005f1c    00000050     lwiplib.obj (.text:netif_add)
                  00005f6c    00000050     lwiplib.obj (.text:sys_timeouts_init)
                  00005fbc    00000050     lwiplib.obj (.text:tcp_write_checks)
                  0000600c    0000004e     lwiplib.obj (.text:autoip_start_probing)
                  0000605a    0000004e     lwiplib.obj (.text:inet_chksum_pbuf)
                  000060a8    0000004e     lwiplib.obj (.text:pbuf_free)
                  000060f6    00000002     --HOLE-- [fill = 0]
                  000060f8    0000004c     lwiplib.obj (.text:ip_route)
                  00006144    0000004c     lwiplib.obj (.text:tivaif_interrupt)
                  00006190    0000004c     lwiplib.obj (.text:udp_connect)
                  000061dc    0000004c     lwiplib.obj (.text:udp_new_port)
                  00006228    00000048     driverlib.lib : sysctl.obj (.text:_SysCtlFrequencyGet)
                  00006270    00000048     enet_tcpecho_server.obj (.text:echo_poll)
                  000062b8    00000048     lwiplib.obj (.text:etharp_output_to_arp_index)
                  00006300    00000048     lwiplib.obj (.text:ip_output)
                  00006348    00000048     lwiplib.obj (.text:tcp_kill_prio)
                  00006390    00000048     lwiplib.obj (.text:tcp_rexmit_fast)
                  000063d8    00000048     lwiplib.obj (.text:tivaif_check_pbuf)
                  00006420    00000046     lwiplib.obj (.text:tcp_send_empty_ack)
                  00006466    00000046     lwiplib.obj (.text:tcp_send_fin)
                  000064ac    00000044     rtsv7M4_T_le_v4SPD16_eabi.lib : autoinit.c.obj (.text:__TI_auto_init_nobinit_nopinit:__TI_auto_init_nobinit_nopinit)
                  000064f0    00000044     lwiplib.obj (.text:tcp_keepalive)
                  00006534    00000042     lwiplib.obj (.text:dhcp_network_changed)
                  00006576    00000042     lwiplib.obj (.text:dhcp_option_long)
                  000065b8    00000042     lwiplib.obj (.text:tcp_pcb_purge)
                  000065fa    00000002     --HOLE-- [fill = 0]
                  000065fc    00000040     lwiplib.obj (.text:etharp_tmr)
                  0000663c    00000040     rtsv7M4_T_le_v4SPD16_eabi.lib : u_divt2.asm.obj (.text)
                  0000667c    0000003e     lwiplib.obj (.text:netif_set_link_up)
                  000066ba    00000002     --HOLE-- [fill = 0]
                  000066bc    0000003c     lwiplib.obj (.text:dhcp_coarse_tmr)
                  000066f8    0000003b     enet_tcpecho_server.obj (.text:echo_sent)
                  00006733    00000001     --HOLE-- [fill = 0]
                  00006734    0000003a     driverlib.lib : emac.obj (.text:EMACIntEnable)
                  0000676e    00000002     --HOLE-- [fill = 0]
                  00006770    00000038     enet_tcpecho_server.obj (.text:DisplayIPAddress)
                  000067a8    00000038     driverlib.lib : emac.obj (.text:EMACConfigSet)
                  000067e0    00000038                   : sysctl.obj (.text:SysCtlPeripheralReady)
                  00006818    00000038     lwiplib.obj (.text:dhcp_fine_tmr)
                  00006850    00000038     lwiplib.obj (.text:dhcp_handle_nak)
                  00006888    00000038     lwiplib.obj (.text:dhcp_stop)
                  000068c0    00000038     lwiplib.obj (.text:memp_free)
                  000068f8    00000038     lwiplib.obj (.text:tcpip_tcp_timer)
                  00006930    00000034     driverlib.lib : emac.obj (.text:EMACConfigGet)
                  00006964    00000034                   : emac.obj (.text:EMACIntClear)
                  00006998    00000034     rtsv7M4_T_le_v4SPD16_eabi.lib : boot_cortex_m.c.obj (.text:_c_int00_noargs:_c_int00_noargs)
                  000069cc    00000034     lwiplib.obj (.text:autoip_arp_probe)
                  00006a00    00000034     enet_tcpecho_server.obj (.text:echo_accept)
                  00006a34    00000034     lwiplib.obj (.text:tcp_kill_timewait)
                  00006a68    00000034     lwiplib.obj (.text:tcp_timer_needed)
                  00006a9c    00000034     lwiplib.obj (.text:tivaif_init)
                  00006ad0    00000032     lwiplib.obj (.text:ip4_addr_isbroadcast)
                  00006b02    00000032     lwiplib.obj (.text:tcp_recved)
                  00006b34    00000030     lwiplib.obj (.text:dhcp_option_trailer)
                  00006b64    00000030     lwiplib.obj (.text:tcp_update_rcv_ann_wnd)
                  00006b94    00000030     lwiplib.obj (.text:udp_remove)
                  00006bc4    0000002e     lwiplib.obj (.text:tcp_rexmit_rto)
                  00006bf2    0000002c     driverlib.lib : emac.obj (.text:EMACIntStatus)
                  00006c1e    0000002c                   : gpio.obj (.text:GPIODirModeSet)
                  00006c4a    00000002     --HOLE-- [fill = 0]
                  00006c4c    0000002c     lwiplib.obj (.text:autoip_arp_announce)
                  00006c78    0000002c     lwiplib.obj (.text:dhcp_handle_offer)
                  00006ca4    0000002c     lwiplib.obj (.text:etharp_request)
                  00006cd0    0000002a     lwiplib.obj (.text:autoip_bind)
                  00006cfa    0000002a     lwiplib.obj (.text:pbuf_cat)
                  00006d24    0000002a     ustdlib.obj (.text:ustrncpy)
                  00006d4e    00000002     --HOLE-- [fill = 0]
                  00006d50    00000028     enet_tcpecho_server.obj (.text:echo_init)
                  00006d78    00000028     lwiplib.obj (.text:etharp_cleanup_netif)
                  00006da0    00000026     driverlib.lib : emac.obj (.text:EMACPHYRead)
                  00006dc6    00000026                   : emac.obj (.text:EMACPHYWrite)
                  00006dec    00000026     lwiplib.obj (.text:dhcp_check)
                  00006e12    00000026     lwiplib.obj (.text:tcp_recv_null)
                  00006e38    00000024     lwiplib.obj (.text:etharp_free_entry)
                  00006e5c    00000024     rtsv7M4_T_le_v4SPD16_eabi.lib : memcmp.c.obj (.text:memcmp)
                  00006e80    00000024     lwiplib.obj (.text:netif_set_up)
                  00006ea4    00000024     lwiplib.obj (.text:tcp_seg_copy)
                  00006ec8    00000022     enet_tcpecho_server.obj (.text:close_conn)
                  00006eea    00000022     lwiplib.obj (.text:dhcp_option_short)
                  00006f0c    00000020     driverlib.lib : sysctl.obj (.text:_SysCtlMemTimingGet)
                  00006f2c    00000020     lwiplib.obj (.text:autoip_handle_arp_conflict)
                  00006f4c    00000020     lwiplib.obj (.text:dhcp_option)
                  00006f6c    00000020     lwiplib.obj (.text:etharp_send_ip)
                  00006f8c    00000020     lwiplib.obj (.text:lwIPTimer)
                  00006fac    00000020     lwiplib.obj (.text:tcp_eff_send_mss)
                  00006fcc    00000020     lwiplib.obj (.text:tcp_tmr)
                  00006fec    00000020     ustdlib.obj (.text:usprintf)
                  0000700c    0000001e     driverlib.lib : emac.obj (.text:EMACAddrGet)
                  0000702a    0000001e     lwiplib.obj (.text:netif_set_down)
                  00007048    0000001c     lwiplib.obj (.text:lwIPLocalIPAddrGet)
                  00007064    0000001c     lwiplib.obj (.text:netif_set_addr)
                  00007080    0000001c     lwiplib.obj (.text:udp_new)
                  0000709c    0000001a     uartstdio.obj (.text:UARTprintf)
                  000070b6    0000001a     lwiplib.obj (.text:autoip_network_changed)
                  000070d0    0000001a     lwiplib.obj (.text:dhcp_arp_reply)
                  000070ea    0000001a     lwiplib.obj (.text:lwip_htonl)
                  00007104    00000018     lwiplib.obj (.text:arp_timer)
                  0000711c    00000018     lwiplib.obj (.text:autoip_timer)
                  00007134    00000018     lwiplib.obj (.text:dhcp_timer_coarse)
                  0000714c    00000018     lwiplib.obj (.text:dhcp_timer_fine)
                  00007164    00000018     lwiplib.obj (.text:pbuf_pool_is_empty)
                  0000717c    00000018     lwiplib.obj (.text:tcp_next_iss)
                  00007194    00000018     lwiplib.obj (.text:tcp_seg_free)
                  000071ac    00000016     driverlib.lib : emac.obj (.text:EMACReset)
                  000071c2    00000016                   : emac.obj (.text:EMACRxEnable)
                  000071d8    00000016                   : emac.obj (.text:EMACTxEnable)
                  000071ee    00000016                   : gpio.obj (.text:GPIOPinTypeEthernetLED)
                  00007204    00000016     lwiplib.obj (.text:dhcp_delete_msg)
                  0000721a    00000016     lwiplib.obj (.text:dhcp_t1_timeout)
                  00007230    00000016     lwiplib.obj (.text:dhcp_t2_timeout)
                  00007246    00000016     lwiplib.obj (.text:pbuf_ref)
                  0000725c    00000014     enet_tcpecho_server.obj (.text:SysTickIntHandler)
                  00007270    00000014     rtsv7M4_T_le_v4SPD16_eabi.lib : strlen.c.obj (.text:strlen)
                  00007284    00000014     lwiplib.obj (.text:sys_arch_unprotect)
                  00007298    00000014     lwiplib.obj (.text:tcp_close)
                  000072ac    00000012     lwiplib.obj (.text:dhcp_option_byte)
                  000072be    00000012     lwiplib.obj (.text:netif_set_link_down)
                  000072d0    00000012     lwiplib.obj (.text:pbuf_clen)
                  000072e2    00000002     --HOLE-- [fill = 0]
                  000072e4    00000010     driverlib.lib : emac.obj (.text:EMACFrameFilterSet)
                  000072f4    00000010                   : interrupt.obj (.text:IntMasterEnable)
                  00007304    00000010     lwiplib.obj (.text:autoip_stop)
                  00007314    00000010     lwiplib.obj (.text:dhcp_set_state)
                  00007324    00000010     lwiplib.obj (.text:inet_chksum)
                  00007334    00000010     lwiplib.obj (.text:lwip_init)
                  00007344    00000010     lwiplib.obj (.text:pbuf_chain)
                  00007354    00000010     lwiplib.obj (.text:sys_arch_protect)
                  00007364    00000010     lwiplib.obj (.text:tcp_segs_free)
                  00007374    0000000e     rtsv7M4_T_le_v4SPD16_eabi.lib : copy_decompress_none.c.obj (.text:decompress:none:__TI_decompress_none)
                  00007382    0000000c     driverlib.lib : cpu.obj (.text:CPUcpsie)
                  0000738e    0000000c     lwiplib.obj (.text:autoip_restart)
                  0000739a    0000000c     rtsv7M4_T_le_v4SPD16_eabi.lib : copy_zero_init.c.obj (.text:decompress:ZI:__TI_zero_init)
                  000073a6    0000000c     lwiplib.obj (.text:lwip_htons)
                  000073b2    00000002     --HOLE-- [fill = 0]
                  000073b4    0000000c     lwiplib.obj (.text:netif_set_default)
                  000073c0    0000000c     lwiplib.obj (.text:netif_set_gw)
                  000073cc    0000000c     lwiplib.obj (.text:netif_set_netmask)
                  000073d8    0000000c     lwiplib.obj (.text:sys_now)
                  000073e4    0000000a     lwiplib.obj (.text:tcp_poll)
                  000073ee    00000008     driverlib.lib : emac.obj (.text:EMACPowerManagementStatusGet)
                  000073f6    00000008                   : emac.obj (.text:EMACTxDMAPollDemand)
                  000073fe    00000008     lwiplib.obj (.text:icmp_dest_unreach)
                  00007406    00000006     driverlib.lib : emac.obj (.text:EMACRxDMADescriptorListSet)
                  0000740c    00000006                   : emac.obj (.text:EMACTimestampIntStatus)
                  00007412    00000006                   : emac.obj (.text:EMACTxDMADescriptorListSet)
                  00007418    00000006     startup_ccs.obj (.text:ResetISR)
                  0000741e    00000006     driverlib.lib : sysctl.obj (.text:SysCtlDelay)
                  00007424    00000006     lwiplib.obj (.text:tcp_abort)
                  0000742a    00000006     lwiplib.obj (.text:tcp_accept_null)
                  00007430    00000006     lwiplib.obj (.text:tcp_err)
                  00007436    00000006     lwiplib.obj (.text:tcp_new)
                  0000743c    00000006     lwiplib.obj (.text:tcp_recv)
                  00007442    00000006     lwiplib.obj (.text:udp_recv)
                  00007448    00000004     rtsv7M4_T_le_v4SPD16_eabi.lib : pre_init.c.obj (.text:_system_pre_init)
                  0000744c    00000004                                   : exit.c.obj (.text:abort:abort)
                  00007450    00000004     lwiplib.obj (.text:tcp_accept)
                  00007454    00000004     lwiplib.obj (.text:tcp_arg)
                  00007458    00000004     lwiplib.obj (.text:tcp_sent)
                  0000745c    00000004     lwiplib.obj (.text:tcp_setprio)

.const     0    00007460    000002dc     
                  00007460    000001b0     driverlib.lib : sysctl.obj (.const:g_pppui32XTALtoVCO)
                  00007610    0000006c                   : sysctl.obj (.const:g_pui32Xtals)
                  0000767c    00000030                   : sysctl.obj (.const:g_sXTALtoMEMTIM)
                  000076ac    00000014                   : interrupt.obj (.const:g_pui32EnRegs)
                  000076c0    00000010     lwiplib.obj (.const:memp_num)
                  000076d0    00000010     lwiplib.obj (.const:memp_sizes)
                  000076e0    00000010     lwiplib.obj (.const:tcp_pcb_lists)
                  000076f0    0000000d     lwiplib.obj (.const:.string:tcp_backoff)
                  000076fd    00000003     --HOLE-- [fill = 0]
                  00007700    0000000c     uartstdio.obj (.const:g_ui32UARTBase)
                  0000770c    0000000c     uartstdio.obj (.const:g_ui32UARTPeriph)
                  00007718    00000008     driverlib.lib : sysctl.obj (.const:g_pui32VCOFrequencies)
                  00007720    00000007     lwiplib.obj (.const:.string:tcp_persist_backoff)
                  00007727    00000006     lwiplib.obj (.const:ethbroadcast)
                  0000772d    00000006     lwiplib.obj (.const:ethzero)
                  00007733    00000001     --HOLE-- [fill = 0]
                  00007734    00000004     lwiplib.obj (.const:ip_addr_any)
                  00007738    00000004     lwiplib.obj (.const:ip_addr_broadcast)

.cinit     0    00007740    00000058     
                  00007740    00000032     (.cinit..data.load) [load image, compression = lzss]
                  00007772    00000002     --HOLE-- [fill = 0]
                  00007774    0000000c     (__TI_handler_table)
                  00007780    00000008     (.cinit..bss.load) [load image, compression = zero_init]
                  00007788    00000010     (__TI_cinit_table)

.init_array 
*          0    00000000    00000000     UNINITIALIZED

.bss       0    20000000    00017a93     UNINITIALIZED
                  20000000    0001001c     (.common:ram_heap)
                  2001001c    000072d4     lwiplib.obj (.bss:memp_memory)
                  200172f0    00000360     (.common:g_pTxDescriptors)
                  20017650    00000120     (.common:g_pRxDescriptors)
                  20017770    00000120     (.common:lwip_stats)
                  20017890    000000c8     lwiplib.obj (.bss:arp_table)
                  20017958    00000050     lwiplib.obj (.bss)
                  200179a8    00000038     lwiplib.obj (.bss:g_sNetIF)
                  200179e0    00000028     (.common:dhcp_rx_options_val)
                  20017a08    00000020     lwiplib.obj (.bss:memp_tab)
                  20017a28    00000010     lwiplib.obj (.bss:inseg)
                  20017a38    0000000c     (.common:dhcp_rx_options_given)
                  20017a44    00000004     (.common:current_header)
                  20017a48    00000004     (.common:current_iphdr_dest)
                  20017a4c    00000004     (.common:current_iphdr_src)
                  20017a50    00000004     (.common:current_netif)
                  20017a54    00000004     (.common:g_pfnTimerHandler)
                  20017a58    00000004     (.common:g_ui32AbnormalInts)
                  20017a5c    00000004     (.common:g_ui32IPAddress)
                  20017a60    00000004     (.common:g_ui32NormalInts)
                  20017a64    00000004     (.common:g_ui32SysClock)
                  20017a68    00000004     (.common:netif_default)
                  20017a6c    00000004     (.common:netif_list)
                  20017a70    00000004     (.common:tcp_active_pcbs)
                  20017a74    00000004     (.common:tcp_bound_pcbs)
                  20017a78    00000004     (.common:tcp_input_pcb)
                  20017a7c    00000004     (.common:tcp_listen_pcbs)
                  20017a80    00000004     (.common:tcp_ticks)
                  20017a84    00000004     (.common:tcp_tmp_pcb)
                  20017a88    00000004     (.common:tcp_tw_pcbs)
                  20017a8c    00000004     (.common:udp_pcbs)
                  20017a90    00000001     (.common:g_bLED)
                  20017a91    00000001     (.common:pbuf_free_ooseq_pending)
                  20017a92    00000001     (.common:tcp_active_pcbs_changed)

.data      0    2001ca98    00001070     UNINITIALIZED
                  2001ca98    00001000     enet_tcpecho_server.obj (.data:g_pctcpBuffer)
                  2001da98    00000038     lwiplib.obj (.data)
                  2001dad0    00000010     lwiplib.obj (.data:g_RxDescList)
                  2001dae0    00000010     lwiplib.obj (.data:g_TxDescList)
                  2001daf0    0000000c     lwiplib.obj (.data:g_StellarisIFData)
                  2001dafc    00000005     uartstdio.obj (.data)
                  2001db01    00000003     --HOLE--
                  2001db04    00000004     enet_tcpecho_server.obj (.data)

.stack     0    20017a98    00005000     UNINITIALIZED
                  20017a98    00000004     rtsv7M4_T_le_v4SPD16_eabi.lib : boot_cortex_m.c.obj (.stack)
                  20017a9c    00004ffc     --HOLE--

__llvm_prf_cnts 
*          0    20000000    00000000     UNINITIALIZED

.binit     0    00000000    00000000     

MODULE SUMMARY

       Module                       code    ro data   rw data
       ------                       ----    -------   -------
    .\
       enet_tcpecho_server.obj      1153    0         4109   
       startup_ccs.obj              12      512       0      
    +--+----------------------------+-------+---------+---------+
       Total:                       1165    512       4109   
                                                             
    .\drivers\
       pinout.obj                   524     0         0      
    +--+----------------------------+-------+---------+---------+
       Total:                       524     0         0      
                                                             
    .\utils\
       lwiplib.obj                  23652   88        97006  
       uartstdio.obj                696     24        5      
       ustdlib.obj                  667     0         0      
    +--+----------------------------+-------+---------+---------+
       Total:                       25015   112       97011  
                                                             
    C:/ti/TivaWare_C_Series-2.2.0.295/driverlib/ccs/Debug/driverlib.lib
       sysctl.obj                   758     596       0      
       emac.obj                     572     0         0      
       gpio.obj                     430     0         0      
       interrupt.obj                120     20        0      
       cpu.obj                      12      0         0      
    +--+----------------------------+-------+---------+---------+
       Total:                       1892    616       0      
                                                             
    C:\ti\ccs1011\ccs\tools\compiler\ti-cgt-arm_20.2.1.LTS\lib\rtsv7M4_T_le_v4SPD16_eabi.lib
       memcpy_t2.asm.obj            156     0         0      
       memset_t2.asm.obj            122     0         0      
       copy_decompress_lzss.c.obj   104     0         0      
       autoinit.c.obj               68      0         0      
       u_divt2.asm.obj              64      0         0      
       boot_cortex_m.c.obj          52      0         0      
       memcmp.c.obj                 36      0         0      
       strlen.c.obj                 20      0         0      
       copy_decompress_none.c.obj   14      0         0      
       copy_zero_init.c.obj         12      0         0      
       exit.c.obj                   4       0         0      
       pre_init.c.obj               4       0         0      
       div0.asm.obj                 2       0         0      
    +--+----------------------------+-------+---------+---------+
       Total:                       658     0         0      
                                                             
       Stack:                       0       0         20480  
       Linker Generated:            0       86        0      
    +--+----------------------------+-------+---------+---------+
       Grand Total:                 29254   1326      121600 


LINKER GENERATED COPY TABLES

__TI_cinit_table @ 00007788 records: 2, size/record: 8, table size: 16
	.data: load addr=00007740, load size=00000032 bytes, run addr=2001ca98, run size=00001070 bytes, compression=lzss
	.bss: load addr=00007780, load size=00000008 bytes, run addr=20000000, run size=00017a93 bytes, compression=zero_init


LINKER GENERATED HANDLER TABLE

__TI_handler_table @ 00007774 records: 3, size/record: 4, table size: 12
	index: 0, handler: __TI_decompress_lzss
	index: 1, handler: __TI_decompress_none
	index: 2, handler: __TI_zero_init


GLOBAL SYMBOLS: SORTED ALPHABETICALLY BY Name 

address   name                          
-------   ----                          
0000744d  C$$EXIT                       
00007383  CPUcpsie                      
00006771  DisplayIPAddress              
0000700d  EMACAddrGet                   
00006931  EMACConfigGet                 
000067a9  EMACConfigSet                 
000072e5  EMACFrameFilterSet            
00006965  EMACIntClear                  
00006735  EMACIntEnable                 
00006bf3  EMACIntStatus                 
00005bc9  EMACPHYConfigSet              
00006da1  EMACPHYRead                   
00006dc7  EMACPHYWrite                  
000073ef  EMACPowerManagementStatusGet  
000071ad  EMACReset                     
00007407  EMACRxDMADescriptorListSet    
000071c3  EMACRxEnable                  
0000740d  EMACTimestampIntStatus        
00007413  EMACTxDMADescriptorListSet    
000073f7  EMACTxDMAPollDemand           
000071d9  EMACTxEnable                  
00006c1f  GPIODirModeSet                
00002955  GPIOPadConfigSet              
000071ef  GPIOPinTypeEthernetLED        
00003ee1  InitDMADescriptors            
00005581  IntEnable                     
000072f5  IntMasterEnable               
00001b21  PinoutSet                     
00007419  ResetISR                      
00001d2d  SysCtlClockFreqSet            
0000741f  SysCtlDelay                   
000067e1  SysCtlPeripheralReady         
00005e7d  SysCtlPeripheralReset         
0000725d  SysTickIntHandler             
000059f5  UARTStdioConfig               
0000709d  UARTprintf                    
00001f2d  UARTvprintf                   
00005ecd  UARTwrite                     
2001ca98  __STACK_END                   
00005000  __STACK_SIZE                  
2001ca98  __STACK_TOP                   
00007788  __TI_CINIT_Base               
00007798  __TI_CINIT_Limit              
00007774  __TI_Handler_Table_Base       
00007780  __TI_Handler_Table_Limit      
000064ad  __TI_auto_init_nobinit_nopinit
000055e9  __TI_decompress_lzss          
00007375  __TI_decompress_none          
ffffffff  __TI_pprof_out_hndl           
ffffffff  __TI_prof_data_size           
ffffffff  __TI_prof_data_start          
00000000  __TI_static_base__            
0000739b  __TI_zero_init                
00004f7b  __aeabi_idiv0                 
00004f7b  __aeabi_ldiv0                 
00005265  __aeabi_memclr                
00005265  __aeabi_memclr4               
00005265  __aeabi_memclr8               
00004761  __aeabi_memcpy                
00004761  __aeabi_memcpy4               
00004761  __aeabi_memcpy8               
00005267  __aeabi_memset                
00005267  __aeabi_memset4               
00005267  __aeabi_memset8               
0000663d  __aeabi_uidiv                 
0000663d  __aeabi_uidivmod              
ffffffff  __binit__                     
ffffffff  __c_args__                    
UNDEFED   __mpu_init                    
20017a98  __stack                       
20000000  __start___llvm_prf_cnts       
20000000  __stop___llvm_prf_cnts        
00006999  _c_int00_noargs               
UNDEFED   _system_post_cinit            
00007449  _system_pre_init              
0000744d  abort                         
00004efd  autoip_arp_reply              
000070b7  autoip_network_changed        
00005c79  autoip_start                  
00007305  autoip_stop                   
00003ad5  autoip_tmr                    
ffffffff  binit                         
20017a44  current_header                
20017a48  current_iphdr_dest            
20017a4c  current_iphdr_src             
20017a50  current_netif                 
000070d1  dhcp_arp_reply                
000066bd  dhcp_coarse_tmr               
00006819  dhcp_fine_tmr                 
00006535  dhcp_network_changed          
00004569  dhcp_release                  
00004cfd  dhcp_renew                    
20017a38  dhcp_rx_options_given         
200179e0  dhcp_rx_options_val           
00004611  dhcp_start                    
00006889  dhcp_stop                     
00006d51  echo_init                     
00006d79  etharp_cleanup_netif          
000030f9  etharp_output                 
00003215  etharp_query                  
000039f9  etharp_raw                    
00006ca5  etharp_request                
000065fd  etharp_tmr                    
00007727  ethbroadcast                  
00004411  ethernet_input                
0000772d  ethzero                       
2001dad0  g_RxDescList                  
2001dae0  g_TxDescList                  
20017a90  g_bLED                        
20017650  g_pRxDescriptors              
200172f0  g_pTxDescriptors              
2001ca98  g_pctcpBuffer                 
20017a54  g_pfnTimerHandler             
00000000  g_pfnVectors                  
20017a58  g_ui32AbnormalInts            
20017a5c  g_ui32IPAddress               
2001da9c  g_ui32LocalTimer              
20017a60  g_ui32NormalInts              
20017a64  g_ui32SysClock                
2001db04  g_ui32tcpPollTick             
000073ff  icmp_dest_unreach             
000027d1  icmp_input                    
00007325  inet_chksum                   
0000605b  inet_chksum_pbuf              
00006ad1  ip4_addr_isbroadcast          
00007734  ip_addr_any                   
00007738  ip_addr_broadcast             
0000211d  ip_input                      
00006301  ip_output                     
000046b9  ip_output_if                  
000060f9  ip_route                      
00004d7d  lwIPEthernetIntHandler        
00004931  lwIPHostTimerHandler          
00003745  lwIPInit                      
00007049  lwIPLocalIPAddrGet            
00006f8d  lwIPTimer                     
000070eb  lwip_htonl                    
000073a7  lwip_htons                    
00007335  lwip_init                     
000070eb  lwip_ntohl                    
000073a7  lwip_ntohs                    
20017770  lwip_stats                    
000024b5  main                          
000053c9  mem_free                      
00005ab5  mem_init                      
0000364d  mem_malloc                    
00003831  mem_trim                      
00006e5d  memcmp                        
00004761  memcpy                        
000068c1  memp_free                     
00005515  memp_init                     
00005cd1  memp_malloc                   
0000526d  memset                        
00005f1d  netif_add                     
20017a68  netif_default                 
20017a6c  netif_list                    
00007065  netif_set_addr                
000073b5  netif_set_default             
0000702b  netif_set_down                
000073c1  netif_set_gw                  
00005721  netif_set_ipaddr              
000072bf  netif_set_link_down           
0000667d  netif_set_link_up             
000073cd  netif_set_netmask             
00006e81  netif_set_up                  
00002e99  pbuf_alloc                    
00006cfb  pbuf_cat                      
00007345  pbuf_chain                    
000072d1  pbuf_clen                     
000049c5  pbuf_copy                     
00005929  pbuf_copy_partial             
000060a9  pbuf_free                     
20017a91  pbuf_free_ooseq_pending       
0000598f  pbuf_header                   
00005b6d  pbuf_realloc                  
00007247  pbuf_ref                      
20000000  ram_heap                      
00005355  raw_input                     
00007271  strlen                        
00007355  sys_arch_protect              
00007285  sys_arch_unprotect            
000073d9  sys_now                       
00005789  sys_timeout                   
00005f6d  sys_timeouts_init             
00004a59  tcp_abandon                   
00007425  tcp_abort                     
00007451  tcp_accept                    
20017a70  tcp_active_pcbs               
20017a92  tcp_active_pcbs_changed       
00003c7d  tcp_alloc                     
00007455  tcp_arg                       
000076f0  tcp_backoff                   
00004e7d  tcp_bind                      
20017a74  tcp_bound_pcbs                
00007299  tcp_close                     
00006fad  tcp_eff_send_mss              
000044bd  tcp_enqueue_flags             
00007431  tcp_err                       
00005439  tcp_fasttmr                   
00000d51  tcp_input                     
20017a78  tcp_input_pcb                 
000064f1  tcp_keepalive                 
20017a7c  tcp_listen_pcbs               
000047fd  tcp_listen_with_backlog       
00007437  tcp_new                       
0000717d  tcp_next_iss                  
00002645  tcp_output                    
000076e0  tcp_pcb_lists                 
000065b9  tcp_pcb_purge                 
00005b11  tcp_pcb_remove                
00007720  tcp_persist_backoff           
000073e5  tcp_poll                      
00005859  tcp_process_refused_data      
0000743d  tcp_recv                      
00006e13  tcp_recv_null                 
00006b03  tcp_recved                    
00005d81  tcp_rexmit                    
00006391  tcp_rexmit_fast               
00006bc5  tcp_rexmit_rto                
0000516d  tcp_rst                       
00006ea5  tcp_seg_copy                  
00007195  tcp_seg_free                  
00007365  tcp_segs_free                 
00006421  tcp_send_empty_ack            
00006467  tcp_send_fin                  
00007459  tcp_sent                      
0000745d  tcp_setprio                   
000013dd  tcp_slowtmr                   
20017a80  tcp_ticks                     
00006a69  tcp_timer_needed              
20017a84  tcp_tmp_pcb                   
00006fcd  tcp_tmr                       
20017a88  tcp_tw_pcbs                   
00006b65  tcp_update_rcv_ann_wnd        
000010f9  tcp_write                     
00004ae9  tcp_zero_window_probe         
00006a9d  tivaif_init                   
00006145  tivaif_interrupt              
000051e9  tivaif_process_phy_interrupt  
000058c1  udp_bind                      
00006191  udp_connect                   
000022f5  udp_input                     
00007081  udp_new                       
20017a8c  udp_pcbs                      
00007443  udp_recv                      
00006b95  udp_remove                    
00004069  udp_sendto_if                 
00006fed  usprintf                      
00006d25  ustrncpy                      
000016a5  uvsnprintf                    


GLOBAL SYMBOLS: SORTED BY Symbol Address 

address   name                          
-------   ----                          
00000000  __TI_static_base__            
00000000  g_pfnVectors                  
00000d51  tcp_input                     
000010f9  tcp_write                     
000013dd  tcp_slowtmr                   
000016a5  uvsnprintf                    
00001b21  PinoutSet                     
00001d2d  SysCtlClockFreqSet            
00001f2d  UARTvprintf                   
0000211d  ip_input                      
000022f5  udp_input                     
000024b5  main                          
00002645  tcp_output                    
000027d1  icmp_input                    
00002955  GPIOPadConfigSet              
00002e99  pbuf_alloc                    
000030f9  etharp_output                 
00003215  etharp_query                  
0000364d  mem_malloc                    
00003745  lwIPInit                      
00003831  mem_trim                      
000039f9  etharp_raw                    
00003ad5  autoip_tmr                    
00003c7d  tcp_alloc                     
00003ee1  InitDMADescriptors            
00004069  udp_sendto_if                 
00004411  ethernet_input                
000044bd  tcp_enqueue_flags             
00004569  dhcp_release                  
00004611  dhcp_start                    
000046b9  ip_output_if                  
00004761  __aeabi_memcpy                
00004761  __aeabi_memcpy4               
00004761  __aeabi_memcpy8               
00004761  memcpy                        
000047fd  tcp_listen_with_backlog       
00004931  lwIPHostTimerHandler          
000049c5  pbuf_copy                     
00004a59  tcp_abandon                   
00004ae9  tcp_zero_window_probe         
00004cfd  dhcp_renew                    
00004d7d  lwIPEthernetIntHandler        
00004e7d  tcp_bind                      
00004efd  autoip_arp_reply              
00004f7b  __aeabi_idiv0                 
00004f7b  __aeabi_ldiv0                 
00005000  __STACK_SIZE                  
0000516d  tcp_rst                       
000051e9  tivaif_process_phy_interrupt  
00005265  __aeabi_memclr                
00005265  __aeabi_memclr4               
00005265  __aeabi_memclr8               
00005267  __aeabi_memset                
00005267  __aeabi_memset4               
00005267  __aeabi_memset8               
0000526d  memset                        
00005355  raw_input                     
000053c9  mem_free                      
00005439  tcp_fasttmr                   
00005515  memp_init                     
00005581  IntEnable                     
000055e9  __TI_decompress_lzss          
00005721  netif_set_ipaddr              
00005789  sys_timeout                   
00005859  tcp_process_refused_data      
000058c1  udp_bind                      
00005929  pbuf_copy_partial             
0000598f  pbuf_header                   
000059f5  UARTStdioConfig               
00005ab5  mem_init                      
00005b11  tcp_pcb_remove                
00005b6d  pbuf_realloc                  
00005bc9  EMACPHYConfigSet              
00005c79  autoip_start                  
00005cd1  memp_malloc                   
00005d81  tcp_rexmit                    
00005e7d  SysCtlPeripheralReset         
00005ecd  UARTwrite                     
00005f1d  netif_add                     
00005f6d  sys_timeouts_init             
0000605b  inet_chksum_pbuf              
000060a9  pbuf_free                     
000060f9  ip_route                      
00006145  tivaif_interrupt              
00006191  udp_connect                   
00006301  ip_output                     
00006391  tcp_rexmit_fast               
00006421  tcp_send_empty_ack            
00006467  tcp_send_fin                  
000064ad  __TI_auto_init_nobinit_nopinit
000064f1  tcp_keepalive                 
00006535  dhcp_network_changed          
000065b9  tcp_pcb_purge                 
000065fd  etharp_tmr                    
0000663d  __aeabi_uidiv                 
0000663d  __aeabi_uidivmod              
0000667d  netif_set_link_up             
000066bd  dhcp_coarse_tmr               
00006735  EMACIntEnable                 
00006771  DisplayIPAddress              
000067a9  EMACConfigSet                 
000067e1  SysCtlPeripheralReady         
00006819  dhcp_fine_tmr                 
00006889  dhcp_stop                     
000068c1  memp_free                     
00006931  EMACConfigGet                 
00006965  EMACIntClear                  
00006999  _c_int00_noargs               
00006a69  tcp_timer_needed              
00006a9d  tivaif_init                   
00006ad1  ip4_addr_isbroadcast          
00006b03  tcp_recved                    
00006b65  tcp_update_rcv_ann_wnd        
00006b95  udp_remove                    
00006bc5  tcp_rexmit_rto                
00006bf3  EMACIntStatus                 
00006c1f  GPIODirModeSet                
00006ca5  etharp_request                
00006cfb  pbuf_cat                      
00006d25  ustrncpy                      
00006d51  echo_init                     
00006d79  etharp_cleanup_netif          
00006da1  EMACPHYRead                   
00006dc7  EMACPHYWrite                  
00006e13  tcp_recv_null                 
00006e5d  memcmp                        
00006e81  netif_set_up                  
00006ea5  tcp_seg_copy                  
00006f8d  lwIPTimer                     
00006fad  tcp_eff_send_mss              
00006fcd  tcp_tmr                       
00006fed  usprintf                      
0000700d  EMACAddrGet                   
0000702b  netif_set_down                
00007049  lwIPLocalIPAddrGet            
00007065  netif_set_addr                
00007081  udp_new                       
0000709d  UARTprintf                    
000070b7  autoip_network_changed        
000070d1  dhcp_arp_reply                
000070eb  lwip_htonl                    
000070eb  lwip_ntohl                    
0000717d  tcp_next_iss                  
00007195  tcp_seg_free                  
000071ad  EMACReset                     
000071c3  EMACRxEnable                  
000071d9  EMACTxEnable                  
000071ef  GPIOPinTypeEthernetLED        
00007247  pbuf_ref                      
0000725d  SysTickIntHandler             
00007271  strlen                        
00007285  sys_arch_unprotect            
00007299  tcp_close                     
000072bf  netif_set_link_down           
000072d1  pbuf_clen                     
000072e5  EMACFrameFilterSet            
000072f5  IntMasterEnable               
00007305  autoip_stop                   
00007325  inet_chksum                   
00007335  lwip_init                     
00007345  pbuf_chain                    
00007355  sys_arch_protect              
00007365  tcp_segs_free                 
00007375  __TI_decompress_none          
00007383  CPUcpsie                      
0000739b  __TI_zero_init                
000073a7  lwip_htons                    
000073a7  lwip_ntohs                    
000073b5  netif_set_default             
000073c1  netif_set_gw                  
000073cd  netif_set_netmask             
000073d9  sys_now                       
000073e5  tcp_poll                      
000073ef  EMACPowerManagementStatusGet  
000073f7  EMACTxDMAPollDemand           
000073ff  icmp_dest_unreach             
00007407  EMACRxDMADescriptorListSet    
0000740d  EMACTimestampIntStatus        
00007413  EMACTxDMADescriptorListSet    
00007419  ResetISR                      
0000741f  SysCtlDelay                   
00007425  tcp_abort                     
00007431  tcp_err                       
00007437  tcp_new                       
0000743d  tcp_recv                      
00007443  udp_recv                      
00007449  _system_pre_init              
0000744d  C$$EXIT                       
0000744d  abort                         
00007451  tcp_accept                    
00007455  tcp_arg                       
00007459  tcp_sent                      
0000745d  tcp_setprio                   
000076e0  tcp_pcb_lists                 
000076f0  tcp_backoff                   
00007720  tcp_persist_backoff           
00007727  ethbroadcast                  
0000772d  ethzero                       
00007734  ip_addr_any                   
00007738  ip_addr_broadcast             
00007774  __TI_Handler_Table_Base       
00007780  __TI_Handler_Table_Limit      
00007788  __TI_CINIT_Base               
00007798  __TI_CINIT_Limit              
20000000  __start___llvm_prf_cnts       
20000000  __stop___llvm_prf_cnts        
20000000  ram_heap                      
200172f0  g_pTxDescriptors              
20017650  g_pRxDescriptors              
20017770  lwip_stats                    
200179e0  dhcp_rx_options_val           
20017a38  dhcp_rx_options_given         
20017a44  current_header                
20017a48  current_iphdr_dest            
20017a4c  current_iphdr_src             
20017a50  current_netif                 
20017a54  g_pfnTimerHandler             
20017a58  g_ui32AbnormalInts            
20017a5c  g_ui32IPAddress               
20017a60  g_ui32NormalInts              
20017a64  g_ui32SysClock                
20017a68  netif_default                 
20017a6c  netif_list                    
20017a70  tcp_active_pcbs               
20017a74  tcp_bound_pcbs                
20017a78  tcp_input_pcb                 
20017a7c  tcp_listen_pcbs               
20017a80  tcp_ticks                     
20017a84  tcp_tmp_pcb                   
20017a88  tcp_tw_pcbs                   
20017a8c  udp_pcbs                      
20017a90  g_bLED                        
20017a91  pbuf_free_ooseq_pending       
20017a92  tcp_active_pcbs_changed       
20017a98  __stack                       
2001ca98  __STACK_END                   
2001ca98  __STACK_TOP                   
2001ca98  g_pctcpBuffer                 
2001da9c  g_ui32LocalTimer              
2001dad0  g_RxDescList                  
2001dae0  g_TxDescList                  
2001db04  g_ui32tcpPollTick             
ffffffff  __TI_pprof_out_hndl           
ffffffff  __TI_prof_data_size           
ffffffff  __TI_prof_data_start          
ffffffff  __binit__                     
ffffffff  __c_args__                    
ffffffff  binit                         
UNDEFED   __mpu_init                    
UNDEFED   _system_post_cinit            

[250 symbols]
